:020000040000FA
:0408000063EF09F0A9
:1008100003B283EF05F0F2B4A1EF05F09EB0A9EFAB
:1008200005F09EB2B1EF05F0F2A81AEF04F0F2B2B3
:1008300032EF04F09EB61FEF04F012EF09F09E961F
:1008400000011450000A06E000011450010A06E0FD
:1008500012EF09F07CEC20F012EF09F074EC22F0BA
:1008600012EF09F0CD90F2929EA03CEF04F001014E
:10087000533F3CEF04F0542BAEC1B2F1AFC1B3F122
:10088000B0C1B4F1B1C1B5F1AAC1AEF1ABC1AFF124
:10089000ACC1B0F1ADC1B1F1A6C1AAF1A7C1ABF134
:1008A000A8C1ACF1A9C1ADF1A2C1A6F1A3C1A7F144
:1008B000A4C1A8F1A5C1A9F19EC1A2F19FC1A3F154
:1008C000A0C1A4F1A1C1A5F19AC19EF19BC19FF164
:1008D0009CC1A0F19DC1A1F196C19AF197C19BF174
:1008E00098C19CF199C19DF1CECF96F1CFCF97F1F0
:1008F00053C198F154C199F1CF6ACE6A0101536B8B
:10090000546B9E90CD800FBC0F8E0FBA8BEF04F00E
:100910000F8A12EF09F00F8C0FBEC7EF04F096C1DB
:100920009AF197C19BF198C19CF199C19DF19AC12F
:100930009EF19BC19FF19CC1A0F19DC1A1F19EC1FF
:10094000A2F19FC1A3F1A0C1A4F1A1C1A5F1A2C1CF
:10095000A6F1A3C1A7F1A4C1A8F1A5C1A9F1A6C19F
:10096000AAF1A7C1ABF1A8C1ACF1A9C1ADF1AAC16F
:10097000AEF1ABC1AFF1ACC1B0F1ADC1B1F1AEC13F
:10098000B2F1AFC1B3F1B0C1B4F1B1C1B5F1010180
:100990005E6B5F6B606B616B96515E2797515F2357
:1009A00098516023995161239A515E279B515F238F
:1009B0009C5160239D5161239E515E279F515F236F
:1009C000A0516023A1516123A2515E27A3515F234F
:1009D000A4516023A5516123A6515E27A7515F232F
:1009E000A8516023A9516123AA515E27AB515F230F
:1009F000AC516023AD516123AE515E27AF515F23EF
:100A0000B0516023B1516123B2515E27B3515F23CE
:100A1000B4516023B5516123D89001016133603333
:100A20005F335E33D8900101613360335F335E33EF
:100A3000D8900101613360335F335E3300C10CF144
:100A400001C10DF102C10EF103C10FF104C110F19A
:100A500005C111F106C112F107C113F108C114F16A
:100A600009C115F10AC116F10BC117F134C135F1F5
:100A700011B846EF05F00101620E046F010E056F1B
:100A8000000E066F000E076F4FEF05F00101A70E75
:100A9000046F020E056F000E066F000E076F5EC139
:100AA00000F15FC101F160C102F161C103F113EC1A
:100AB0001FF003BF04D019BE02D019A0108C11A0E2
:100AC00067EF05F010BA67EF05F00F80108A0CC1D0
:100AD00000F10DC101F10EC102F10FC103F110C10E
:100AE00004F111C105F112C106F113C107F114C1DE
:100AF00008F115C109F116C10AF117C10BF135C191
:100B000034F112EF09F00392ABB2AB98AB8803015A
:100B100003EE00F080517F0BE92604C0EFFF802B2D
:100B20008151805D700BD8A48B8200008051815D63
:100B3000700BD8A48B9281518019D8B4079012EF12
:100B400009F0F2940101453F12EF09F0462B12EF34
:100B500009F09E900101533F12EF09F0542B12EF60
:100B600009F09E9211B820EF07F08BB4BFEF05F0AB
:100B700010ACBFEF05F08B84109CC0EF05F08B9498
:100B8000C3CF55F1C4CF56F1C28207B42AEF06F0A5
:100B900047C14BF148C14CF149C14DF14AC14EF139
:100BA0005EC162F15FC163F160C164F161C165F171
:100BB00096C1B6F197C1B7F198C1B8F199C1B9F131
:100BC0009AC1BAF19BC1BBF19CC1BCF19DC1BDF101
:100BD0009EC1BEF19FC1BFF1A0C1C0F1A1C1C1F1D1
:100BE000A2C1C2F1A3C1C3F1A4C1C4F1A5C1C5F1A1
:100BF000A6C1C6F1A7C1C7F1A8C1C8F1A9C1C9F171
:100C0000AAC1CAF1ABC1CBF1ACC1CCF1ADC1CDF140
:100C1000AEC1CEF1AFC1CFF1B0C1D0F1B1C1D1F110
:100C2000B2C1D2F1B3C1D3F1B4C1D4F1B5C1D5F1E0
:100C3000010155515B2756515C23E86A5D230E2E56
:100C40002AEF06F05CC157F15DC158F15B6B5C6B3C
:100C50005D6B078E0201002F12EF09F03C0E006F52
:100C60001A50E00BE00AE866128818BE02D018B4E9
:100C7000108E00C10CF101C10DF102C10EF103C1D2
:100C80000FF104C110F105C111F106C112F107C144
:100C900013F108C114F109C115F10AC116F10BC114
:100CA00017F134C135F101018A675EEF06F08B67F9
:100CB0005EEF06F08C675EEF06F08D6762EF06F080
:100CC00092EF06F08EC100F18FC101F190C102F1E7
:100CD00091C103F10101010E046F000E056F000EBA
:100CE000066F000E076F13EC1FF000C18EF101C1FB
:100CF0008FF102C190F103C191F1006787EF06F017
:100D0000016787EF06F0026787EF06F0036792EF4F
:100D100006F08AC18EF18BC18FF18CC190F18DC12B
:100D200091F10F80D57ED5BE6DD0D6CF47F1D7CF0C
:100D300048F145C149F1E86AE8CF4AF119BE02D04D
:100D400019A0108C109047C100F148C101F149C1B0
:100D500002F14AC103F101010A0E046F000E056F92
:100D6000000E066F000E076F13EC1FF003AF10802C
:100D7000010154A7C8EF06F00F9A0F9C0F9E0101C6
:100D8000000E5E6F600E5F6F3D0E606F080E616F4C
:100D9000010147BFD8EF06F04867D8EF06F0496772
:100DA000D8EF06F04A67D8EF06F0F288FDEF06F0BC
:100DB000F2985E6B5F6B606B616B966B976B986B79
:100DC000996B9A6B9B6B9C6B9D6B9E6B9F6BA06BE7
:100DD000A16BA26BA36BA46BA56BA66BA76BA86B97
:100DE000A96BAA6BAB6BAC6BAD6BAE6BAF6BB06B47
:100DF000B16BB26BB36BB46BB56BD76AD66A0101DA
:100E0000456B466B0CC100F10DC101F10EC102F141
:100E10000FC103F110C104F111C105F112C106F1B6
:100E200013C107F114C108F115C109F116C10AF186
:100E300017C10BF135C134F112EF09F012EF09F0CF
:100E40000201002F79EF08F0D59ED6CF47F1D7CF1A
:100E500048F145C149F1E86AE8CF4AF1D76AD66A54
:100E60000101456B466BD58E1A50E00BE00AE8662F
:100E7000128818BE02D018B4108E17AE1C8C00C198
:100E80000CF101C10DF102C10EF103C10FF104C15A
:100E900010F105C111F106C112F107C113F108C12A
:100EA00014F109C115F10AC116F10BC117F134C1D2
:100EB00035F10FA0109A11B869EF07F00101620E29
:100EC000046F010E056F000E066F000E076F72EFC4
:100ED00007F00101A70E046F020E056F000E066FEA
:100EE000000E076F47C100F148C101F149C102F18D
:100EF0004AC103F113EC1FF003BF85EF07F019BEE1
:100F000002D019A0108C11B00F800CC100F10DC1DE
:100F100001F10EC102F10FC103F110C104F111C1C1
:100F200005F112C106F113C107F114C108F115C191
:100F300009F116C10AF117C10BF135C134F10201F3
:100F40003C0E006F00C10CF101C10DF102C10EF1A8
:100F500003C10FF104C110F105C111F106C112F175
:100F600007C113F108C114F109C115F10AC116F145
:100F70000BC117F134C135F101018A67C7EF07F0E2
:100F80008B67C7EF07F08C67C7EF07F08D67CBEF74
:100F900007F0FBEF07F08EC100F18FC101F190C1A6
:100FA00002F191C103F10101010E046F000E056F02
:100FB000000E066F000E076F13EC1FF000C18EF1DC
:100FC00001C18FF102C190F103C191F10067F0EF0F
:100FD00007F00167F0EF07F00267F0EF07F0036733
:100FE000FBEF07F08AC18EF18BC18FF18CC190F1BC
:100FF0008DC191F10F80109047C100F148C101F1FE
:1010000049C102F14AC103F101010A0E046F000E49
:10101000056F000E066F000E076F13EC1FF003AF95
:101020001080010154A721EF08F00F9A0F9C0F9E2A
:101030000101000E5E6F600E5F6F3D0E606F080E67
:10104000616F47C100F148C101F149C102F14AC1D4
:1010500003F10101140E046F050E056F000E066FFB
:10106000000E076F13EC1FF003AF3AEF08F0F288A1
:101070005FEF08F0F2985E6B5F6B606B616B966B75
:10108000976B986B996B9A6B9B6B9C6B9D6B9E6B34
:101090009F6BA06BA16BA26BA36BA46BA56BA66BE4
:1010A000A76BA86BA96BAA6BAB6BAC6BAD6BAE6B94
:1010B000AF6BB06BB16BB26BB36BB46BB56B0CC198
:1010C00000F10DC101F10EC102F10FC103F110C118
:1010D00004F111C105F112C106F113C107F114C1E8
:1010E00008F115C109F116C10AF117C10BF135C19B
:1010F00034F133EC23F01D661ED01CAE11D01C9EC3
:101100001D8E18AE07D0146A040E156E166A7CEC9C
:1011100020F011D0146A156A166A7CEC20F00BD00E
:101120001CAC09D01C9C1D8C010E146E156A166A2D
:1011300074EC22F000D08BB4A5EF08F010ACA5EF52
:1011400008F08B84109CA6EF08F08B94C3CF55F168
:10115000C4CF56F1C28207B410EF09F047C14BF17A
:1011600048C14CF149C14DF14AC14EF15EC162F135
:101170005FC163F160C164F161C165F196C1B6F10F
:1011800097C1B7F198C1B8F199C1B9F19AC1BAF153
:101190009BC1BBF19CC1BCF19DC1BDF19EC1BEF123
:1011A0009FC1BFF1A0C1C0F1A1C1C1F1A2C1C2F1F3
:1011B000A3C1C3F1A4C1C4F1A5C1C5F1A6C1C6F1C3
:1011C000A7C1C7F1A8C1C8F1A9C1C9F1AAC1CAF193
:1011D000ABC1CBF1ACC1CCF1ADC1CDF1AEC1CEF163
:1011E000AFC1CFF1B0C1D0F1B1C1D1F1B2C1D2F133
:1011F000B3C1D3F1B4C1D4F1B5C1D5F10101555199
:101200005B2756515C23E86A5D230E2E10EF09F030
:101210005CC157F15DC158F15B6B5C6B5D6B078E18
:1012200012EF09F002C0E0FF005001C0D8FF10002B
:10123000A6B218EF09F00CC0A9FF0BC0A8FFA69E2C
:10124000A69CA684F29E550EA76EAA0EA76EA68235
:10125000F28EA694A6B22AEF09F00C2A1200A96E0B
:10126000A69EA69CA680A8500C2A120004012C0E53
:10127000826F3BEC0BF00EEC20F00C502FEC09F0E1
:10128000E8CF00F10C502FEC09F0E8CF01F101AFED
:101290004FEF09F00101FF0E026FFF0E036FB1EC7B
:1012A0001FF029675BEF09F00401200E826F3BEC11
:1012B0000BF060EF09F004012D0E826F3BEC0BF098
:1012C000BBEC1DF01200306A076A0F6A106A116ADF
:1012D000126A136A0F010E0EC16E860EC06E030EE7
:1012E000C26E0F01896A110E926E080E8A6EF10E9F
:1012F000936E8B6A980E946EF18EFC0E2FEC09F0B3
:10130000E8CF0BF00BA011800BA211820BA411846B
:101310000BA81188C90E2FEC09F0E8CF17F0CA0E00
:101320002FEC09F0E8CF18F0CB0E2FEC09F0E8CF46
:1013300019F0CC0E2FEC09F0E8CF1AF0CD0E2FECFF
:1013400009F0E8CF2FF01C6A1D6A0E6A01015B6B81
:101350005C6B5D6B576B586BF29A0101476B486B86
:10136000496B4A6B4B6B4C6B4D6B4E6B4F6B506BC1
:10137000516B526B456B466BD76AD66A0F01280ECC
:10138000D56EF28A9D90B00ECD6E01015E6B5F6BE3
:10139000606B616B626B636B646B656B666B676BD9
:1013A000686B696B536B546BCF6ACE6A0F9A0F9C54
:1013B0000F9E9D80760ECA6E9D8202013C0E006FCC
:1013C000CC6A160E2FEC09F0E8CF00F1170E2FECC7
:1013D00009F0E8CF01F1180E2FEC09F0E8CF02F187
:1013E000190E2FEC09F0E8CF03F1010103AF13EF61
:1013F0000AF00EEC20F0160E0C6E00C10BF018EC8B
:1014000009F0170E0C6E01C10BF018EC09F0180E64
:101410000C6E02C10BF018EC09F0190E0C6E03C132
:101420000BF018EC09F000C18AF101C18BF102C187
:101430008CF103C18DF100C18EF101C18FF102C1A8
:1014400090F103C191F11A0E2FEC09F0E8CF00F1F1
:101450001B0E2FEC09F0E8CF01F11C0E2FEC09F068
:10146000E8CF02F11D0E2FEC09F0E8CF03F10101E6
:1014700003AF69EF0AF00EEC20F01A0E0C6E00C1FB
:101480000BF018EC09F01B0E0C6E01C10BF018EC00
:1014900009F01C0E0C6E02C10BF018EC09F01D0EC9
:1014A0000C6E03C10BF018EC09F01A0E2FEC09F0CA
:1014B000E8CF00F11B0E2FEC09F0E8CF01F11C0E74
:1014C0002FEC09F0E8CF02F11D0E2FEC09F0E8CF68
:1014D00003F100C192F101C193F102C194F103C182
:1014E00095F1240EAC6E900EAB6E240EAC6E080E11
:1014F000B86E000EB06E1F0EAF6E0401806B816B74
:101500000F01900EAB6E0F019D8A0301806B816B02
:10151000C26B8B92146A156A166A9D860790000149
:10152000F28EF28C07B064EF1CF00FB0FCEF15F0F8
:1015300010BEFCEF15F012B8FCEF15F0030180515E
:1015400081197F0BD8B464EF1CF013EE00F08151C9
:101550007F0BE126812BE7CFE8FFE00BD8B464EFE7
:101560001CF023EE82F0C2513F0BD926E7CFDFFFFC
:10157000C22BDF50780AD8A464EF1CF007808EC11C
:1015800000F18FC101F190C102F191C103F101019C
:10159000040E046F000E056F000E066F000E076F3D
:1015A00013EC1FF000AFDEEF0AF00101030E8E6FA7
:1015B000000E8F6F000E906F000E916F030182512D
:1015C000720AD8B4E1EF15F08251520AD8B4E1EFB3
:1015D00015F08251750AD8B4E1EF15F08251630A13
:1015E000D8B41EEF19F08251690AD8B488EF12F00E
:1015F00082517A0AD8B49BEF13F08251490AD8B4C9
:1016000027EF12F08251500AD8B431EF11F0825115
:10161000700AD8B479EF11F08251540AD8B4A9EF06
:1016200011F08251740AD8B4F4EF11F08251410ADA
:10163000D8B451EF0CF082514B0AD8B44FEF0BF0F5
:1016400082516D0AD8B484EF10F082514D0AD8B49B
:101650009DEF10F08251730AD8B411EF15F082514A
:10166000530AD8B476EF15F08251590AD8B4D5EFA1
:101670000FF055EF19F0040114EE00F080517F0BCC
:10168000E12682C4E7FF802B120004010D0E826F59
:101690003BEC0BF00A0E826F3BEC0BF012000401E6
:1016A0004B0E826F3BEC0BF004012C0E826F3BEC77
:1016B0000BF081B802D02FB630D003018351430A1A
:1016C000D8B494EF0BF003018351630AD8B496EFBA
:1016D0000BF003018351520AD8B498EF0BF00301C9
:1016E0008351720AD8B49AEF0BF003018351470A71
:1016F000D8B49CEF0BF003018351670AD8B49EEF76
:101700000BF003018351540AD8B4A0EF0BF003018E
:101710008351740AD8B40FEF0CF003018351550ABA
:10172000D8B4A2EF0BF082D02F807AD02F9078D04F
:101730002F8276D02F9274D02F8472D02F9470D0B5
:101740002F866ED084C330F185C331F186C332F168
:1017500087C333F10101296B5CEC20F0D3EC1FF05F
:1017600000C104F101C105F102C106F103C107F195
:101770004FEC20F0200EF86EF76AF66A0900F5CFFC
:101780002CF10900F5CF2DF10900F5CF2EF109005C
:10179000F5CF2FF10900F5CF30F10900F5CF31F188
:1017A0000900F5CF32F10900F5CF33F10101296BC2
:1017B0005CEC20F0D3EC1FF013EC1FF00067E8EFB7
:1017C0000BF00167E8EF0BF00267E8EF0BF003673F
:1017D00001D025D004014E0E826F3BEC0BF00401CA
:1017E0006F0E826F3BEC0BF004014D0E826F3BECF1
:1017F0000BF00401610E826F3BEC0BF00401740EE0
:10180000826F3BEC0BF00401630E826F3BEC0BF03C
:101810000401680E826F3BEC0BF053EF19F02F962A
:10182000CD0E0C6E2FC00BF018EC09F0CD0E2FEC86
:1018300009F0E8CF2FF02FB006D00401630E826FBD
:101840003BEC0BF005D00401430E826F3BEC0BF038
:101850002FB206D00401720E826F3BEC0BF005D064
:101860000401520E826F3BEC0BF02FB406D0040142
:10187000670E826F3BEC0BF005D00401470E826FC0
:101880003BEC0BF02FB606D00401740E826F3BECDC
:101890000BF005D00401540E826F3BEC0BF053EFBC
:1018A00019F00401410E826F3BEC0BF003018351F0
:1018B000310AD8B4F5EF0EF003018351320AD8B4DF
:1018C00025EF0EF003018351330AD8B4AEEF0DF0CB
:1018D00003018351340AD8B49EEF0CF00301835105
:1018E000350AD8B47BEF0CF004013F0E826F3BEC5D
:1018F0000BF053EF19F004012C0E826F3BEC0BF050
:1019000003018451300AD8B48EEF0CF003018451E6
:10191000310AD8B496EF0CF0E7EF0DF08B9004018C
:10192000300E826F3BEC0BF09CEF0CF08B800401CF
:10193000310E826F3BEC0BF053EF19F0CC0E2FEC15
:1019400009F0E8CF0BF004012C0E826F3BEC0BF09A
:1019500003018451310AD8B4C2EF0CF00301845161
:10196000300AD8B4C4EF0CF0030184514D0AD8B446
:10197000CEEF0CF003018451540AD8B4D5EF0CF02B
:10198000ECEF0CF08A8401D08A940BAE04D00BAC3F
:1019900002D00BBA21D0E00E0B1218D01F0E0B167E
:1019A0008539E844E00B0B1211D0E00E0B164FEC1A
:1019B00020F085C332F186C333F10101296B5CEC61
:1019C00020F0D3EC1FF000511F0B0B12CC0E0C6E4D
:1019D0000BC00BF018EC09F00401340E826F3BECE5
:1019E0000BF004012C0E826F3BEC0BF0CC0E2FECB5
:1019F00009F0E8CF1AF08AB406D00401300E826FE5
:101A00003BEC0BF005D00401310E826F3BEC0BF088
:101A100004012C0E826F3BEC0BF01A38E840070BE8
:101A2000E8CF82F40401300E82273BEC0BF0040176
:101A30002C0E826F3BEC0BF00EEC20F01A501F0BBB
:101A4000E8CF00F1B1EC1FF032C182F40401300E96
:101A500082273BEC0BF033C182F40401300E822765
:101A60003BEC0BF004012C0E826F3BEC0BF00EEC08
:101A700020F02DC000F100AF0BD0FF0E016FFF0E64
:101A8000026FFF0E036F04012D0E826F3BEC0BF013
:101A9000B1EC1FF031C182F40401300E82273BEC1F
:101AA0000BF032C182F40401300E82273BEC0BF0C4
:101AB00033C182F40401300E82273BEC0BF00401A9
:101AC0002C0E826F3BEC0BF00EEC20F02CC000F1E2
:101AD000B1EC1FF031C182F40401300E82273BECDF
:101AE0000BF032C182F40401300E82273BEC0BF084
:101AF00033C182F40401300E82273BEC0BF0040169
:101B00002C0E826F3BEC0BF00EEC20F02EC000F19F
:101B100000AF0BD0FF0E016FFF0E026FFF0E036FC1
:101B200004012D0E826F3BEC0BF0B1EC1FF031C1C4
:101B300082F40401300E82273BEC0BF032C182F4B8
:101B40000401300E82273BEC0BF033C182F4040118
:101B5000300E82273BEC0BF053EF19F0CB0E2FEC3D
:101B600009F0E8CF0BF004012C0E826F3BEC0BF078
:101B700003018451450AD8B4D2EF0DF0030184511A
:101B8000440AD8B4D5EF0DF003018451300AD8B41B
:101B9000D8EF0DF003018451310AD8B4DCEF0DF019
:101BA000E7EF0DF00B9EE1EF0DF00B8EE1EF0DF086
:101BB000FC0E0B16E1EF0DF0FC0E0B160B80E1EFA7
:101BC0000DF0CB0E0C6E0BC00BF018EC09F00401FD
:101BD000330E826F3BEC0BF004012C0E826F3BEC5A
:101BE0000BF0CB0E2FEC09F0E8CF19F019BE00EF87
:101BF0000EF00401450E826F3BEC0BF005EF0EF08A
:101C00000401440E826F3BEC0BF004012C0E826F3A
:101C10003BEC0BF00401300E826F3BEC0BF0040147
:101C20002C0E826F3BEC0BF019B01EEF0EF004018E
:101C3000300E826F3BEC0BF023EF0EF00401310EFF
:101C4000826F3BEC0BF053EF19F0CA0E2FEC09F04A
:101C5000E8CF0BF004012C0E826F3BEC0BF003017C
:101C60008451450AD8B461EF0EF003018451440A4F
:101C7000D8B464EF0EF0030184514D0AD8B46DEF6F
:101C80000EF003018451410AD8B467EF0EF003014E
:101C90008451460AD8B46AEF0EF003018451560A03
:101CA000D8B475EF0EF003018451500AD8B480EF18
:101CB0000EF003018451520AD8B483EF0EF08CEF7A
:101CC0000EF00B9E86EF0EF00B8E86EF0EF00B9C47
:101CD00086EF0EF00B8C86EF0EF0FC0E0B1685C314
:101CE000E8FF030B0B1286EF0EF0C70E0B1685C331
:101CF000E8FF070BE846E846E8460B1286EF0EF0D1
:101D00000B8486EF0EF00B9486EF0EF0CA0E0C6E6D
:101D10000BC00BF018EC09F0CA0E2FEC09F0E8CF5D
:101D200018F00401320E826F3BEC0BF004012C0E14
:101D3000826F3BEC0BF018BEA5EF0EF00401450ED0
:101D4000826F3BEC0BF0AAEF0EF00401440E826FA1
:101D50003BEC0BF004012C0E826F3BEC0BF018C037
:101D6000E8FF030BE8CF82F40401300E82273BEC3E
:101D70000BF004012C0E826F3BEC0BF018BCC8EF8B
:101D80000EF00401410E826F3BEC0BF0CDEF0EF034
:101D90000401460E826F3BEC0BF004012C0E826FA7
:101DA0003BEC0BF018C0E8FF380BE842E842E84291
:101DB000E8CF82F40401300E82273BEC0BF00401E3
:101DC0002C0E826F3BEC0BF018B4EEEF0EF004011A
:101DD000520E826F3BEC0BF0F3EF0EF00401500E4D
:101DE000826F3BEC0BF053EF19F0C90E2FEC09F0AA
:101DF000E8CF0BF004012C0E826F3BEC0BF00301DB
:101E00008451450AD8B413EF0FF003018451440AFA
:101E1000D8B416EF0FF0030184514D0AD8B419EF6E
:101E20000FF027EF0FF00B9E21EF0FF00B8E21EF3D
:101E30000FF0F80E0B1685C3E8FF070B0B1221EF0E
:101E40000FF0C90E0C6E0BC00BF018EC09F004017A
:101E5000310E826F3BEC0BF004012C0E826F3BECD9
:101E60000BF0C90E2FEC09F0E8CF17F017BE06D023
:101E70000401450E826F3BEC0BF005D00401440ECB
:101E8000826F3BEC0BF004012C0E826F3BEC0BF0ED
:101E900017C0E8FF070BE8CF82F40401300E822759
:101EA0003BEC0BF004012C0E826F3BEC0BF0078037
:101EB0000EEC20F028C0E8FF003B00430043030B7A
:101EC000B1EC1FF033C182F40401300E82273BECE9
:101ED0000BF004012C0E826F3BEC0BF00EEC20F0AB
:101EE00028C001F1019F019D29C000F10101B1EC61
:101EF0001FF02FC182F40401300E82273BEC0BF05F
:101F000030C182F40401300E82273BEC0BF031C16A
:101F100082F40401300E82273BEC0BF032C182F4D4
:101F20000401300E82273BEC0BF033C182F4040134
:101F3000300E82273BEC0BF004012C0E826F3BEC41
:101F40000BF00EEC20F02AC001F12BC000F1D8906C
:101F500001330033D890013300330101B1EC1FF09D
:101F60002FC182F40401300E82273BEC0BF030C10C
:101F700082F40401300E82273BEC0BF031C182F475
:101F80000401300E82273BEC0BF032C182F40401D5
:101F9000300E82273BEC0BF033C182F40401300E8B
:101FA00082273BEC0BF053EF19F0FC0E2FEC09F0FD
:101FB000E8CF0BF003018351520AD8B40CEF10F0B4
:101FC00003018351720AD8B40FEF10F0030183515B
:101FD000500AD8B412EF10F003018351700AD8B43C
:101FE00015EF10F003018351550AD8B418EF10F023
:101FF00003018351750AD8B41BEF10F0030183511C
:10200000430AD8B424EF10F003018351630AD8B413
:1020100027EF10F030EF10F00B902AEF10F00B804C
:102020002AEF10F00B922AEF10F00B822AEF10F03B
:102030000B942AEF10F00B842AEF10F00B962AEF86
:1020400010F00B862AEF10F00B982AEF10F00B8897
:102050002AEF10F0FC0E0C6E0BC00BF018EC09F020
:102060000401590E826F3BEC0BF011901192119408
:102070001198FC0E2FEC09F0E8CF0BF00BA01180AB
:102080000BA211820BA411840BA8118811A050EF90
:1020900010F00401520E826F3BEC0BF055EF10F084
:1020A0000401720E826F3BEC0BF011A85FEF10F091
:1020B0000401430E826F3BEC0BF064EF10F004015F
:1020C000630E826F3BEC0BF011A26EEF10F0040177
:1020D000500E826F3BEC0BF073EF10F00401700EAA
:1020E000826F3BEC0BF011A47DEF10F00401550E54
:1020F000826F3BEC0BF082EF10F00401750E826FE3
:102100003BEC0BF053EF19F004016D0E826F3BECCA
:102110000BF003018351300AD8B4E1EF10F0030152
:102120008351310AD8B4F4EF10F003018351320A1D
:10213000D8B407EF11F055EF19F081B803D02FB4E0
:1021400053EF19F004014D0E826F3BEC0BF04FEC96
:1021500020F084C331F185C332F186C333F101012C
:10216000296B5CEC20F0D3EC1FF003018351300AA3
:10217000D8B4C9EF10F003018351310AD8B4D1EFBC
:1021800010F003018351320AD8B4D9EF10F055EFA3
:1021900019F0FD0E0C6E00C10BF018EC09F0E1EF28
:1021A00010F0FE0E0C6E00C10BF018EC09F0F4EF0D
:1021B00010F0FF0E0C6E00C10BF018EC09F007EFE9
:1021C00011F00401300E826F3BEC0BF004012C0E79
:1021D000826F3BEC0BF00EEC20F0FD0E2FEC09F0C3
:1021E000E8CF00F118EF11F00401310E826F3BECE3
:1021F0000BF004012C0E826F3BEC0BF00EEC20F088
:10220000FE0E2FEC09F0E8CF00F118EF11F00401F9
:10221000320E826F3BEC0BF00EEC20F004012C0E22
:10222000826F3BEC0BF0FF0E2FEC09F0E8CF00F1D2
:10223000B1EC1FF031C182F40401300E82273BEC77
:102240000BF032C182F40401300E82273BEC0BF01C
:1022500033C182F40401300E82273BEC0BF053EFC4
:1022600019F081B803D02FB227EF12F083C32AF1FF
:1022700084C32BF185C32CF186C32DF187C32EF1C6
:1022800088C32FF189C330F18AC331F18BC332F196
:102290008CC333F101015CEC20F0D3EC1FF0160E7F
:1022A0000C6E00C10BF018EC09F0170E0C6E01C19A
:1022B0000BF018EC09F0180E0C6E02C10BF018ECC4
:1022C00009F0190E0C6E03C10BF018EC09F000C1F7
:1022D0008AF101C18BF102C18CF103C18DF100C102
:1022E0008EF101C18FF102C190F103C191F127EF8D
:1022F00012F081B803D02FB227EF12F083C32AF176
:1023000084C32BF185C32CF186C32DF187C32EF135
:1023100088C32FF189C330F18AC331F18BC332F105
:102320008CC333F101015CEC20F0D3EC1FF000C151
:102330008AF101C18BF102C18CF103C18DF100C1A1
:102340008EF101C18FF102C190F103C191F127EF2C
:1023500012F081B803D02FB227EF12F083C32AF115
:1023600084C32BF185C32CF186C32DF187C32EF1D5
:1023700088C32FF189C330F18AC331F18CC332F1A4
:102380008DC333F101015CEC20F0D3EC1FF00101AF
:10239000000E046F000E056F010E066F000E076F32
:1023A00024EC1FF01A0E0C6E00C10BF018EC09F0B3
:1023B0001B0E0C6E01C10BF018EC09F01C0E0C6E1C
:1023C00002C10BF018EC09F01D0E0C6E03C10BF0EE
:1023D00018EC09F000C192F101C193F102C194F12E
:1023E00003C195F127EF12F081B803D02FB227EF88
:1023F00012F083C32AF184C32BF185C32CF186C369
:102400002DF187C32EF188C32FF189C330F18AC320
:1024100031F18CC332F18DC333F101015CEC20F05A
:10242000D3EC1FF00101000E046F000E056F010ECA
:10243000066F000E076F24EC1FF000C192F101C17E
:1024400093F102C194F103C195F127EF12F0160E3A
:102450002FEC09F0E8CF00F1170E2FEC09F0E8CFD0
:1024600001F1180E2FEC09F0E8CF02F1190E2FEC54
:1024700009F0E8CF03F1B1EC1FF074EC1DF004019A
:10248000730E826F3BEC0BF004012C0E826F3BEC61
:102490000BF08AC100F18BC101F18CC102F18DC139
:1024A00003F1B1EC1FF074EC1DF00401730E826FA8
:1024B0003BEC0BF004012C0E826F3BEC0BF01A0E80
:1024C0002FEC09F0E8CF00F11B0E2FEC09F0E8CF5C
:1024D00001F11C0E2FEC09F0E8CF02F11D0E2FECDC
:1024E00009F0E8CF03F170EC19F004012C0E826FB3
:1024F0003BEC0BF092C100F193C101F194C102F1E8
:1025000095C103F170EC19F045EC0BF055EF19F0A3
:102510000401690E826F3BEC0BF004012C0E826FFC
:102520003BEC0BF00101040E006F000E016F000E7A
:10253000026F000E036FB1EC1FF02CC182F4040196
:10254000300E82273BEC0BF02DC182F40401300EDB
:1025500082273BEC0BF02EC182F40401300E82275F
:102560003BEC0BF02FC182F40401300E82273BECD0
:102570000BF030C182F40401300E82273BEC0BF0EB
:1025800031C182F40401300E82273BEC0BF032C1E2
:1025900082F40401300E82273BEC0BF033C182F44D
:1025A0000401300E82273BEC0BF004012C0E826FED
:1025B0003BEC0BF00101030E006F000E016F000EEB
:1025C000026F000E036FB1EC1FF02CC182F4040106
:1025D000300E82273BEC0BF02DC182F40401300E4B
:1025E00082273BEC0BF02EC182F40401300E8227CF
:1025F0003BEC0BF02FC182F40401300E82273BEC40
:102600000BF030C182F40401300E82273BEC0BF05A
:1026100031C182F40401300E82273BEC0BF032C151
:1026200082F40401300E82273BEC0BF033C182F4BC
:102630000401300E82273BEC0BF004012C0E826F5C
:102640003BEC0BF00101360E006F000E016F000E27
:10265000026F000E036FB1EC1FF02CC182F4040175
:10266000300E82273BEC0BF02DC182F40401300EBA
:1026700082273BEC0BF02EC182F40401300E82273E
:102680003BEC0BF02FC182F40401300E82273BECAF
:102690000BF030C182F40401300E82273BEC0BF0CA
:1026A00031C182F40401300E82273BEC0BF032C1C1
:1026B00082F40401300E82273BEC0BF033C182F42C
:1026C0000401300E82273BEC0BF004012C0E826FCC
:1026D0003BEC0BF0200EF86EF76AF66A0401090075
:1026E000F5CF82F43BEC0BF00900F5CF82F43BEC24
:1026F0000BF00900F5CF82F43BEC0BF00900F5CFAD
:1027000082F43BEC0BF00900F5CF82F43BEC0BF0CC
:102710000900F5CF82F43BEC0BF00900F5CF82F411
:102720003BEC0BF00900F5CF82F43BEC0BF045ECF1
:102730000BF055EF19F081B803D02FB0EBEF13F089
:102740008351630AD8A453EF19F08451610AD8A4C5
:1027500053EF19F085516C0AD8A453EF19F0865144
:10276000410A42E08651440A1BE08651420AD8B42D
:1027700007EF14F08651350AD8B4DFEF1AF086510E
:10278000360AD8B434EF1BF08651370AD8B49DEF1F
:102790001BF08651380AD8B4FBEF1BF053EF19F049
:1027A0000798079A04017A0E826F3BEC0BF0040144
:1027B000780E826F3BEC0BF00401640E826F3BECF1
:1027C0000BF081A8EBEF13F00401550E826F3BEC88
:1027D0000BF0F0EF13F004014C0E826F3BEC0BF0AA
:1027E00045EC0BF055EF19F00788079A04017A0EB3
:1027F000826F3BEC0BF00401410E826F3BEC0BF05F
:102800000401610E826F3BEC0BF0E1EF13F00798CF
:10281000078A04017A0E826F3BEC0BF00401420E32
:10282000826F3BEC0BF00401610E826F3BEC0BF00E
:10283000E1EF13F00101666725EF14F0676725EFFC
:1028400014F0686725EF14F0696715D04F6730EF13
:1028500014F0506730EF14F0516730EF14F0526706
:102860000AD00101000E006F000E016F000E026F12
:10287000000E036F120011B80AD00101620E046F3E
:10288000010E056F000E066F000E076F09D00101E3
:10289000A70E046F020E056F000E066F000E076F85
:1028A00066C100F167C101F168C102F169C103F1BC
:1028B00013EC1FF003BFCDEF14F0119A119C01012E
:1028C000000E046FA80E056F550E066F020E076FFF
:1028D00066C100F167C101F168C102F169C103F18C
:1028E00066C186F167C187F168C188F169C189F164
:1028F00013EC1FF003BF0BD00101000E866FA80E72
:10290000876F550E886F020E896F118A119C0E0E0B
:102910002FEC09F0E8CF18F10F0E2FEC09F0E8CFFB
:1029200019F1100E2FEC09F0E8CF1AF1110E2FEC6F
:1029300009F0E8CF1BF15CEC1EF086C104F187C101
:1029400005F188C106F189C107F113EC1FF0078278
:1029500020EC1EF05CEC1EF0079220EC1EF086C10D
:1029600000F187C101F188C102F189C103F1079229
:1029700020EC1EF0CC0E046FE00E056F870E066F84
:10298000050E076F13EC1FF000C118F101C119F11A
:1029900002C11AF103C11BF13BD0119C119A010134
:1029A000800E006F1A0E016F060E026F000E036F8D
:1029B0004FC104F150C105F151C106F152C107F1F7
:1029C00013EC1FF003AF05D00EEC20F0118C119A20
:1029D00012000E0E2FEC09F0E8CF18F10F0E2FECBD
:1029E00009F0E8CF19F1100E2FEC09F0E8CF1AF139
:1029F000110E2FEC09F0E8CF1BF14FC100F150C1CF
:102A000001F151C102F152C103F1078220EC1EF025
:102A100018C100F119C101F11AC102F11BC103F182
:102A200012000401730E826F3BEC0BF004012C0EBC
:102A3000826F3BEC0BF0078462C166F163C167F102
:102A400064C168F165C169F14BC14FF14CC150F1EE
:102A50004DC151F14EC152F157C159F158C15AF10E
:102A6000079437EC15F045EC0BF055EF19F066C103
:102A700000F167C101F168C102F169C103F101010F
:102A8000B1EC1FF074EC1DF00401630E826F3BEC9F
:102A90000BF004012C0E826F3BEC0BF04FC100F1E8
:102AA00050C101F151C102F152C103F10101B1EC78
:102AB0001FF074EC1DF00401660E826F3BEC0BF00E
:102AC00004012C0E826F3BEC0BF00EEC20F059C190
:102AD00000F15AC101F10101B1EC1FF074EC1DF0DD
:102AE0000401740E826F3BEC0BF0120010820401A3
:102AF000530E826F3BEC0BF004012C0E826F3BEC0B
:102B00000BF083C32AF184C32BF185C32CF186C358
:102B10002DF187C32EF188C32FF189C330F18AC309
:102B200031F18BC332F18CC333F101015CEC20F045
:102B3000D3EC1FF000C166F101C167F102C168F179
:102B400003C169F18EC32AF18FC32BF190C32CF11D
:102B500091C32DF192C32EF193C32FF194C330F1A1
:102B600095C331F196C332F197C333F101015CECA7
:102B700020F0D3EC1FF000C14FF101C150F102C1B0
:102B800051F103C152F14FEC20F099C32FF19AC3D8
:102B900030F19BC331F19CC332F19DC333F101018C
:102BA0005CEC20F0D3EC1FF000C159F101C15AF1E7
:102BB00037EC15F004012C0E826F3BEC0BF0F0EFBC
:102BC00015F0118E19A002D019AE108C18BE02D0CB
:102BD00018A4108E8251520A02E10F8201D00F9286
:102BE0008251750A02E1108401D010948251550A75
:102BF00002E1108601D0109611A003D011A401D0DB
:102C00001084078410B25EEF16F010A44AEF16F09D
:102C1000B6C166F1B7C167F1B8C168F1B9C169F170
:102C2000BAC16AF1BBC16BF1BCC16CF1BDC16DF140
:102C3000BEC16EF1BFC16FF1C0C170F1C1C171F110
:102C4000C2C172F1C3C173F1C4C174F1C5C175F1E0
:102C5000C6C176F1C7C177F1C8C178F1C9C179F1B0
:102C6000CAC17AF1CBC17BF1CCC17CF1CDC17DF180
:102C7000CEC17EF1CFC17FF1D0C180F1D1C181F150
:102C8000D2C182F1D3C183F1D4C184F1D5C185F120
:102C900052EF16F062C166F163C167F164C168F179
:102CA00065C169F14BC14FF14CC150F14DC151F1BA
:102CB0004EC152F157C159F158C15AF107940FA0B2
:102CC00080EF16F0010192676DEF16F093676DEFDC
:102CD00016F094676DEF16F0956771EF16F080EFC0
:102CE00016F01AEC14F092C104F193C105F194C1ED
:102CF00006F195C107F113EC1FF003BF1BEF19F0AC
:102D00001AEC14F00101000E046F000E056F010EA5
:102D1000066F000E076F44EC1FF011A02AD011A21D
:102D200028D0B1EC1FF0296701D005D004012D0E89
:102D3000826F3BEC0BF030C182F40401300E82272D
:102D40003BEC0BF031C182F40401300E82273BECE6
:102D50000BF032C182F40401300E82273BEC0BF001
:102D600033C182F40401300E82273BEC0BF045ECBA
:102D70000BF012A8C3D012981AC01BF01B3A1B42CA
:102D8000070E1B1600011B50000AD8B44CEF17F0B9
:102D900000011B50010AD8B4D8EF16F000011B50F7
:102DA000020AD8B4D6EF16F07EEF17F07EEF17F0D8
:102DB0000EEC20F02AC001F12BC000F1D8900133B5
:102DC0000033D890013300330101630E046F000E0D
:102DD000056F000E066F000E076F44EC1FF0280E03
:102DE000046F000E056F000E066F000E076F13ECE8
:102DF0001FF000C12DF00EEC20F028C001F1019F62
:102E0000019D29C000F10101A40E046F000E056FA1
:102E1000000E066F000E076F44EC1FF000C12CF08F
:102E200000C104F101C105F102C106F103C107F1BE
:102E3000640E006F000E016F000E026F000E036F34
:102E400013EC1FF0050E046F000E056F000E066FE9
:102E5000000E076F44EC1FF000C104F101C105F141
:102E600002C106F103C107F10EEC20F02DC000F104
:102E700013EC1FF000C12EF02EC0E8FF050F2D5CF3
:102E800003E78A847EEF17F02EC0E8FF0A0F2D5C5F
:102E900001E68A947EEF17F000C124F101C125F10B
:102EA00002C126F103C127F10EEC20F014EC20F052
:102EB0001A501F0BE8CF00F10101640E046F000EE1
:102EC000056F000E066F000E076F24EC1FF024C183
:102ED00004F125C105F126C106F127C107F113EC64
:102EE0001FF003BF02D08A9401D08A8424C100F16C
:102EF00025C101F126C102F127C103F100C124F16E
:102F000001C125F102C126F103C127F110AE4DD058
:102F1000109E00C108F101C109F102C10AF103C10B
:102F20000BF1B1EC1FF030C1D6F131C1D7F132C194
:102F3000D8F133C1D9F108C100F109C101F10AC1C9
:102F400002F10BC103F101016C0E046F070E056F56
:102F5000000E066F000E076F13EC1FF003BF04D0C6
:102F60000101550EDA6F1CD008C100F109C101F151
:102F70000AC102F10BC103F10101A40E046F060E98
:102F8000056F000E066F000E076F13EC1FF003BFF6
:102F900004D001017F0EDA6F03D00101FF0EDA6F5A
:102FA0001C8E11AE1BEF19F0119E24C100F125C13A
:102FB00001F126C102F127C103F111A005D011A230
:102FC00003D00FB01BEF19F010A4EEEF17F00401BF
:102FD000750E826F3BEC0BF0F3EF17F00401720EED
:102FE000826F3BEC0BF004012C0E826F3BEC0BF07C
:102FF000B1EC1FF0296702EF18F00401200E826F78
:1030000005EF18F004012D0E826F3BEC0BF030C180
:1030100082F40401300E82273BEC0BF031C182F4C4
:103020000401300E82273BEC0BF004012E0E826F60
:103030003BEC0BF032C182F40401300E82273BECF2
:103040000BF033C182F40401300E82273BEC0BF00D
:1030500004016D0E826F3BEC0BF004012C0E826FAD
:103060003BEC0BF04FC100F150C101F151C102F135
:1030700052C103F10101B1EC1FF074EC1DF0040129
:10308000480E826F3BEC0BF004017A0E826F3BEC32
:103090000BF004012C0E826F3BEC0BF066C100F1CB
:1030A00067C101F168C102F169C103F10101B1EC2D
:1030B0001FF074EC1DF00401630E826F3BEC0BF00B
:1030C00004012C0E826F3BEC0BF066C100F167C16E
:1030D00001F168C102F169C103F101010A0E046F37
:1030E000000E056F000E066F000E076F24EC1FF038
:1030F000000E046F120E056F000E066F000E076FB4
:1031000044EC1FF0B1EC1FF02AC182F40401300E30
:1031100082273BEC0BF02BC182F40401300E822796
:103120003BEC0BF02CC182F40401300E82273BEC07
:103130000BF02DC182F40401300E82273BEC0BF022
:103140002EC182F40401300E82273BEC0BF02FC11C
:1031500082F40401300E82273BEC0BF030C182F484
:103160000401300E82273BEC0BF004012E0E826F1F
:103170003BEC0BF031C182F40401300E82273BECB2
:103180000BF032C182F40401300E82273BEC0BF0CD
:1031900033C182F40401300E82273BEC0BF00401B2
:1031A000730E826F3BEC0BF004012C0E826F3BEC34
:1031B0000BF00EEC20F059C100F15AC101F17FEC87
:1031C0001AF00FB2E7EF18F00FA019EF19F0040191
:1031D0002C0E826F3BEC0BF0200EF86EF76AF66A4D
:1031E00004010900F5CF82F43BEC0BF00900F5CFA8
:1031F00082F43BEC0BF00900F5CF82F43BEC0BF0D2
:103200000900F5CF82F43BEC0BF00900F5CF82F416
:103210003BEC0BF00900F5CF82F43BEC0BF009001E
:10322000F5CF82F43BEC0BF00900F5CF82F43BECD8
:103230000BF045EC0BF00F9055EF19F00401630E05
:10324000826F3BEC0BF004012C0E826F3BEC0BF019
:103250005BEC19F004012C0E826F3BEC0BF0CEEC12
:1032600019F004012C0E826F3BEC0BF04AEC1AF0C3
:1032700004012C0E826F3BEC0BF00101F80E006F85
:10328000CD0E016F660E026F030E036F70EC19F026
:1032900004012C0E826F3BEC0BF060EC1AF045EC55
:1032A0000BF055EF19F045EC0BF00301C26B0790E2
:1032B000109264EF1CF0D8900E0E2FEC09F0E8CFBE
:1032C00000F10F0E2FEC09F0E8CF01F1100E2FECFA
:1032D00009F0E8CF02F1110E2FEC09F0E8CF03F16D
:1032E0000101000E046F000E056F010E066F000E47
:1032F000076F44EC1FF0B1EC1FF02AC182F4040107
:10330000300E82273BEC0BF02BC182F40401300E0F
:1033100082273BEC0BF02CC182F40401300E822793
:103320003BEC0BF02DC182F40401300E82273BEC04
:103330000BF02EC182F40401300E82273BEC0BF01F
:103340002FC182F40401300E82273BEC0BF030C118
:1033500082F40401300E82273BEC0BF031C182F481
:103360000401300E82273BEC0BF004012E0E826F1D
:103370003BEC0BF032C182F40401300E82273BECAF
:103380000BF033C182F40401300E82273BEC0BF0CA
:1033900004016D0E826F3BEC0BF01200120E2FEC4D
:1033A00009F0E8CF00F1130E2FEC09F0E8CF01F19E
:1033B000140E2FEC09F0E8CF02F1150E2FEC09F0F6
:1033C000E8CF03F101010A0E046F000E056F000E35
:1033D000066F000E076F24EC1FF0000E046F120E34
:1033E000056F000E066F000E076F44EC1FF0B1EC86
:1033F0001FF02AC182F40401300E82273BEC0BF04F
:103400002BC182F40401300E82273BEC0BF02CC15F
:1034100082F40401300E82273BEC0BF02DC182F4C4
:103420000401300E82273BEC0BF02EC182F4040124
:10343000300E82273BEC0BF02FC182F40401300EDA
:1034400082273BEC0BF030C182F40401300E82275E
:103450003BEC0BF004012E0E826F3BEC0BF031C104
:1034600082F40401300E82273BEC0BF032C182F46F
:103470000401300E82273BEC0BF033C182F40401CF
:10348000300E82273BEC0BF00401730E826F3BEC95
:103490000BF012000A0E2FEC09F0E8CF00F10B0E32
:1034A0002FEC09F0E8CF01F10C0E2FEC09F0E8CF7A
:1034B00002F10D0E2FEC09F0E8CF03F17FEF1AF0C7
:1034C000060E2FEC09F0E8CF00F1070E2FEC09F003
:1034D000E8CF01F1080E2FEC09F0E8CF02F1090E58
:1034E0002FEC09F0E8CF03F17FEF1AF001010EECA9
:1034F00020F0078457C100F158C101F10794010180
:10350000E80E046F800E056F000E066F000E076F49
:1035100024EC1FF0000E046F040E056F000E066F02
:10352000000E076F44EC1FF0880E046F130E056F3A
:10353000000E066F000E076F13EC1FF00A0E046FEB
:10354000000E056F000E066F000E076F44EC1FF0B3
:10355000B1EC1FF001012967B3EF1AF00401200E4E
:10356000826FB6EF1AF004012D0E826F3BEC0BF068
:1035700030C182F40401300E82273BEC0BF031C1E4
:1035800082F40401300E82273BEC0BF032C182F44E
:103590000401300E82273BEC0BF004012E0E826FEB
:1035A0003BEC0BF033C182F40401300E82273BEC7C
:1035B0000BF00401430E826F3BEC0BF0120087C34B
:1035C0002AF188C32BF189C32CF18AC32DF18BC357
:1035D0002EF18CC32FF18DC330F18EC331F190C326
:1035E00032F191C333F10101296B5CEC20F0D3EC93
:1035F0001FF00101000E046F000E056F010E066F33
:10360000000E076F24EC1FF00E0E0C6E00C10BF0C5
:1036100018EC09F00F0E0C6E01C10BF018EC09F05C
:10362000100E0C6E02C10BF018EC09F0110E0C6EAE
:1036300003C10BF018EC09F004017A0E826F3BEC29
:103640000BF004012C0E826F3BEC0BF00401350EE5
:10365000826F3BEC0BF004012C0E826F3BEC0BF005
:103660005BEC19F0F0EF13F087C32AF188C32BF15C
:1036700089C32CF18AC32DF18BC32EF18CC32FF19A
:103680008DC330F18EC331F190C332F191C333F168
:103690000101296B5CEC20F0D3EC1FF0880E046F65
:1036A000130E056F000E066F000E076F18EC1FF06B
:1036B000000E046F040E056F000E066F000E076FFC
:1036C00024EC1FF00101E80E046F800E056F000E60
:1036D000066F000E076F44EC1FF00A0E0C6E00C15F
:1036E0000BF018EC09F00B0E0C6E01C10BF018EC8E
:1036F00009F00C0E0C6E02C10BF018EC09F00D0E67
:103700000C6E03C10BF018EC09F004017A0E826F05
:103710003BEC0BF004012C0E826F3BEC0BF0040130
:10372000360E826F3BEC0BF004012C0E826F3BECEB
:103730000BF04AEC1AF0F0EF13F087C32AF188C3BC
:103740002BF189C32CF18AC32DF18BC32EF18CC3CD
:103750002FF18DC330F18FC331F190C332F191C39A
:1037600033F101015CEC20F0D3EC1FF0000E046F8C
:10377000120E056F000E066F000E076F24EC1FF08F
:1037800001010A0E046F000E056F000E066F000E99
:10379000076F44EC1FF0120E0C6E00C10BF018EC1A
:1037A00009F0130E0C6E01C10BF018EC09F0140EA9
:1037B0000C6E02C10BF018EC09F0150E0C6E03C173
:1037C0000BF018EC09F004017A0E826F3BEC0BF061
:1037D00004012C0E826F3BEC0BF00401370E826F5C
:1037E0003BEC0BF004012C0E826F3BEC0BF0CEECAB
:1037F00019F0F0EF13F087C32AF188C32BF189C3C6
:103800002CF18AC32DF18BC32EF18CC32FF18DC304
:1038100030F18EC331F190C332F191C333F1010124
:10382000296B5CEC20F0D3EC1FF0880E046F130EB4
:10383000056F000E066F000E076F18EC1FF0000EEC
:10384000046F040E056F000E066F000E076F24EC68
:103850001FF00101E80E046F800E056F000E066F69
:10386000000E076F44EC1FF0060E0C6E00C10BF04B
:1038700018EC09F0070E0C6E01C10BF018EC09F002
:10388000080E0C6E02C10BF018EC09F0090E0C6E5C
:1038900003C10BF018EC09F004017A0E826F3BECC7
:1038A0000BF004012C0E826F3BEC0BF00401380E80
:1038B000826F3BEC0BF004012C0E826F3BEC0BF0A3
:1038C00060EC1AF0F0EF13F081B803D02FB022EFC4
:1038D0001DF007A8DCEF1CF00101800E006F1A0E2E
:1038E000016F060E026F000E036F4BC104F14CC155
:1038F00005F14DC106F14EC107F113EC1FF003BFF6
:1039000022EF1DF06EEC1DF04BC100F14CC101F136
:103910004DC102F14EC103F1078220EC1EF018C127
:1039200004F119C105F11AC106F11BC107F1F80E26
:10393000006FCD0E016F660E026F030E036F13EC66
:103940001FF00E0E0C6E00C10BF018EC09F00F0EFC
:103950000C6E01C10BF018EC09F0100E0C6E02C1D8
:103960000BF018EC09F0110E0C6E03C10BF018EC03
:1039700009F0078401010EEC20F057C100F158C195
:1039800001F107940A0E0C6E00C10BF018EC09F05F
:103990000B0E0C6E01C10BF018EC09F00C0E0C6E46
:1039A00002C10BF018EC09F00D0E0C6E03C10BF008
:1039B00018EC09F022EF1DF007AA22EF1DF0078492
:1039C00001010EEC20F057C100F158C101F107943C
:1039D000060E0C6E00C10BF018EC09F0070E0C6E11
:1039E00001C10BF018EC09F0080E0C6E02C10BF0CF
:1039F00018EC09F0090E0C6E03C10BF018EC09F07D
:103A0000078462C100F163C101F164C102F165C1C3
:103A100003F10794120E0C6E00C10BF018EC09F0C4
:103A2000130E0C6E01C10BF018EC09F0140E0C6EA5
:103A300002C10BF018EC09F0150E0C6E03C10BF06F
:103A400018EC09F00798079A0401805181197F0B3F
:103A50000DE09EA8FED714EE00F081517F0BE12609
:103A6000E750812B0F01AD6E24EF1DF092EF0AF0AD
:103A700018C100F119C101F11AC102F11BC103F112
:103A8000000E046F000E056F010E066F000E076F2B
:103A900044EC1FF029A163EF1DF02051D8B463EF6F
:103AA0001DF018C100F119C101F11AC102F11BC1C9
:103AB00003F1000E046F000E056F0A0E066F000E74
:103AC000076F44EC1FF0120001010451001305516F
:103AD0000113065102130751031312000101186B61
:103AE000196B1A6B1B6B12002AC182F40401300E91
:103AF00082273BEC0BF02BC182F40401300E8227AD
:103B00003BEC0BF02CC182F40401300E82273BEC1D
:103B10000BF02DC182F40401300E82273BEC0BF038
:103B20002EC182F40401300E82273BEC0BF02FC132
:103B300082F40401300E82273BEC0BF030C182F49A
:103B40000401300E82273BEC0BF031C182F40401FA
:103B5000300E82273BEC0BF032C182F40401300EB0
:103B600082273BEC0BF033C182F40401300E822734
:103B70003BEC0BF012002FC182F40401300E8227BF
:103B80003BEC0BF030C182F40401300E82273BEC99
:103B90000BF031C182F40401300E82273BEC0BF0B4
:103BA00032C182F40401300E82273BEC0BF033C1AA
:103BB00082F40401300E82273BEC0BF01200060E5B
:103BC0001E6E060E1F6E060E206E1E2EE5EF1DF0F9
:103BD0001F2EE5EF1DF0202EE5EF1DF08B84020E69
:103BE0001E6E020E1F6E020E206E1E2EF5EF1DF0D1
:103BF0001F2EF5EF1DF0202EF5EF1DF08B94120017
:103C0000FF0E1F6E1FC020F0030E1E6E8B841E2E33
:103C100006EF1EF0030E1E6E202E06EF1EF08B9494
:103C20001FC020F0030E1E6E1E2E14EF1EF0030E9A
:103C30001E6E203E14EF1EF01F2E02EF1EF012002B
:103C40000101005305E1015303E1025301E1002B9F
:103C5000E3EC1EF00EEC20F03951006F3A51016F89
:103C6000420E046F4B0E056F000E066F000E076FBD
:103C700024EC1FF000C104F101C105F102C106F1FD
:103C800003C107F118C100F119C101F11AC102F114
:103C90001BC103F107B251EF1EF018EC1FF053EFF8
:103CA0001EF013EC1FF000C118F101C119F102C19F
:103CB0001AF103C11BF112000EEC20F059C100F102
:103CC0005AC101F1060E2FEC09F0E8CF04F1070EFE
:103CD0002FEC09F0E8CF05F1080E2FEC09F0E8CF42
:103CE00006F1090E2FEC09F0E8CF07F113EC1FF0F5
:103CF00000C124F101C125F102C126F103C127F160
:103D0000290E046F000E056F000E066F000E076F80
:103D100024EC1FF0EE0E046F430E056F000E066FCD
:103D2000000E076F18EC1FF024C104F125C105F146
:103D300026C106F127C107F124EC1FF000C11CF1D8
:103D400001C11DF102C11EF103C11FF1120E2FECC2
:103D500009F0E8CF04F1130E2FEC09F0E8CF05F1DC
:103D6000140E2FEC09F0E8CF06F1150E2FEC09F038
:103D7000E8CF07F10D0E006F000E016F000E026F0D
:103D8000000E036F24EC1FF0180E046F000E056F79
:103D9000000E066F000E076F44EC1FF01CC104F10B
:103DA0001DC105F11EC106F11FC107F118EC1FF07E
:103DB0006A0E046F2A0E056F000E066F000E076F65
:103DC00013EC1FF01200BF0EFA6E200E3A6F396B23
:103DD000D8900037013702370337D8B0F4EF1EF020
:103DE0003A2FE9EF1EF039073A070353D8B412000F
:103DF0000331070B80093F6F03390F0B010F396F38
:103E000080EC5FF0406F390580EC5FF0405D405F13
:103E1000396B3F33D8B0392739333FA909EF1FF049
:103E2000405139271200010133EC20F0D8B01200C4
:103E3000010103510719346FF6EC1FF0D8900751B8
:103E4000031934AF800F12000101346B1AEC20F01B
:103E5000D8A030EC20F0D8B0120005EC20F00EEC29
:103E600020F01F0E366F46EC20F00B35D8B0F6EC84
:103E70001FF0D8A00335D8B01200362F33EF1FF053
:103E800034B11DEC20F012000101346B0451051116
:103E9000061107110008D8A01AEC20F0D8A030ECC9
:103EA00020F0D8B01200086B096B0A6B0B6B46EC64
:103EB00020F01F0E366F46EC20F007510B5DD8A4A2
:103EC0006EEF1FF006510A5DD8A46EEF1FF005518A
:103ED000095DD8A46EEF1FF00451085DD8A081EFF2
:103EE0001FF00451085F0551D8A0053D095F065138
:103EF000D8A0063D0A5F0751D8A0073D0B5FD890B8
:103F00000081362F5BEF1FF034B11DEC20F0346BD5
:103F10001AEC20F0D8904AEC20F007510B5DD8A4A1
:103F20009EEF1FF006510A5DD8A49EEF1FF00551C9
:103F3000095DD8A49EEF1FF00451085DD8A0ADEF35
:103F40001FF0003FADEF1FF0013FADEF1FF0023F4C
:103F5000ADEF1FF0032BD8B4120034B11DEC20F0EC
:103F600012000101346B1AEC20F0D8B012004FECB3
:103F700020F0200E366F003701370237033711EE7D
:103F800033F00A0E376FE7360A0EE75CD8B0E76EFB
:103F9000E552372FC3EF1FF0362FBBEF1FF034B1C0
:103FA0002981D890120001010A0E346F200E366F5D
:103FB00011EE29F03451376F0A0ED890E652D8B07E
:103FC000E726E732372FDEEF1FF0033302330133EA
:103FD0000033362FD8EF1FF0E750FF0FD8A003357E
:103FE000D8B0120029B11DEC20F0120004510027B6
:103FF0000551D8B0053D01270651D8B0063D02272E
:104000000751D8B0073D032712000051086F015136
:10401000096F02510A6F03510B6F12000101006B0F
:10402000016B026B036B12000101046B056B066BE5
:10403000076B12000335D8A012000351800B001F3C
:10404000011F021F031F003F2DEF20F0013F2DEF46
:1040500020F0023F2DEF20F0032B342B032512001C
:104060000735D8A012000751800B041F051F061F3B
:10407000071F043F43EF20F0053F43EF20F0063FCA
:1040800043EF20F0072B342B0725120000370137B0
:1040900002370337083709370A370B371200010197
:1040A000296B2A6B2B6B2C6B2D6B2E6B2F6B306B54
:1040B000316B326B336B120001012A510F0B2A6FE7
:1040C0002B510F0B2B6F2C510F0B2C6F2D510F0BF6
:1040D0002D6F2E510F0B2E6F2F510F0B2F6F305155
:1040E0000F0B306F31510F0B316F32510F0B326F9D
:1040F00033510F0B336F120000011650FF0A01E11C
:104100001200390EC86E800EC76E280EC66E000EE5
:10411000C56E1550000AD8B4B7EF20F01550010A4B
:10412000D8B4D0EF20F01550020AD8B4E9EF20F04F
:104130001550030AD8B402EF21F01550040AD8B480
:104140002AEF21F01550050AD8B443EF21F015509D
:10415000060AD8B45CEF21F01550070AD8B475EF01
:1041600021F01550080AD8B48EEF21F01200165035
:10417000000AD8B4ADEF21F01650010AD8B4B1EF5F
:1041800021F01650020AD8B4B5EF21F01650030AF8
:10419000D8B4B9EF21F01650040AD8B42CEF22F0AD
:1041A0001650000AD8B4C1EF21F01650010AD8B455
:1041B000C5EF21F01650020AD8B4C9EF21F016500D
:1041C000030AD8B4CDEF21F01650040AD8B42CEF6E
:1041D00022F01650000AD8B4D1EF21F01650010A8F
:1041E000D8B4D5EF21F01650020AD8B4D9EF21F097
:1041F0001650030AD8B4DDEF21F01650040AD8B4E3
:104200002CEF22F01650000AD8B4EAEF21F0165035
:10421000010AD8B4EEEF21F01650020AD8B4F2EF3A
:1042200021F01650030AD8B406EF22F01650040A03
:10423000D8B40AEF22F01650050AD8B40EEF22F0D7
:104240001650060AD8B412EF22F01650070AD8B456
:1042500015EF22F01650000AD8B419EF22F01650CC
:10426000010AD8B41DEF22F01650020AD8B421EF8B
:1042700022F01650030AD8B425EF22F01650040A93
:10428000D8B428EF22F01650000AD8B430EF22F04C
:104290001650010AD8B434EF22F01650020AD8B4EE
:1042A00038EF22F01650030AD8B43CEF22F0165033
:1042B000040AD8B42CEF22F01650000AD8B446EF06
:1042C00022F01650010AD8B44AEF22F01650020A22
:1042D000D8B44EEF22F01650030AD8B452EF22F0B1
:1042E0001650040AD8B42CEF22F01650000AD8B4A5
:1042F00053EF22F01650010AD8B457EF22F01650AF
:10430000020AD8B45BEF22F01650030AD8B45FEF6C
:1043100022F01650040AD8B42CEF22F01650000AEE
:10432000D8B460EF22F01650010AD8B464EF22F03E
:104330001650020AD8B468EF22F01650030AD8B417
:104340006CEF22F01650040AD8B46DEF22F016502C
:10435000050AD8B470EF22F012009E96C580162A86
:104360001200E20EC96E162A1200770EC96E162AC6
:104370001200020EE86E8AB4E88AE8CFC9FF162A56
:1043800012009E96C580162A1200E20EC96E162AE9
:104390001200790EC96E162A1200000EC96E162A76
:1043A00012009E96C580162A1200E20EC96E162AC9
:1043B00012007A0EC96E162A120018BC03D0DAC198
:1043C000E8FF04D01850E844E8441F09E8CFC9FFCB
:1043D000162A12009E96C580162A1200E20EC96E99
:1043E000162A120011BA03D011BC01D003D0050E59
:1043F000156E3ED00101D66702EF22F0100EC96E95
:1044000004EF22F0D6C1C9FF162A1200D7C1C9FF96
:10441000162A1200D8C1C9FF162A1200D9C1C9FF35
:10442000162A1200C584162A1200FF0E166E1D9E53
:1044300012009E96C580162A1200E20EC96E162A38
:104440001200760EC96E162A1200C584162A1200B2
:10445000FF0E166E1D9E1200C584152A166A1200E4
:104460009E96C580162A1200E20EC96E162A120008
:104470007B0EC96E162A120011AA04D0230EC96E33
:10448000162A12001C0EC96E162A12009E96C580AE
:10449000162A1200E20EC96E162A12007C0EC96E90
:1044A000162A1200E9D79E96C580162A1200E20E3F
:1044B000C96E162A12007D0EC96E162A1200DCD7AC
:1044C0009E96C580162A1200E20EC96E162A1200A8
:1044D0007E0EC96E162A1200CFD7C584162A120086
:1044E000FF0E166E1D9E12001650FF0AD8B432EF52
:1044F00023F0390EC86E800EC76E280EC66E000EF1
:10450000C56E1550000AD8B48DEF22F01550010A7F
:10451000D8B4A1EF22F032EF23F01650000AD8B43D
:10452000DFEF22F01650010AD8B4E3EF22F0165064
:10453000020AD8B4EDEF22F01650030AD8B4F0EF17
:1045400022F01650000AD8B4F6EF22F01650010AF5
:10455000D8B4FAEF22F01650020AD8B404EF23F0D0
:104560001650030AD8B407EF23F01650040AD8B443
:104570000DEF23F01650050AD8B410EF23F01650B3
:10458000060AD8B416EF23F01650070AD8B419EF6C
:1045900023F01650080AD8B41FEF23F01650090A6A
:1045A000D8B422EF23F016500A0AD8B428EF23F02B
:1045B00016500B0AD8B42BEF23F032EF23F09E965F
:1045C000C58031EF23F017B004D04E0EC96E31EF25
:1045D00023F0500EC96E31EF23F0C58431EF23F084
:1045E000152AFF0E166E128032EF23F09E96C580BC
:1045F00031EF23F017B004D04F0EC96E31EF23F026
:10460000510EC96E31EF23F0C58631EF23F0C9CFCB
:1046100024F0C59AC58831EF23F0C58631EF23F029
:10462000C9CF25F0C59AC58831EF23F0C58631EF93
:1046300023F0C9CF26F0C59AC58831EF23F0C5868F
:1046400031EF23F0C9CF27F0C58AC58831EF23F0B9
:10465000C58431EF23F0FF0E166E12861D9C32EFDB
:1046600023F0162A120012B012D012B213D012B4D4
:1046700014D012A6120007B01200129624C028F01F
:1046800025C029F026C02AF027C02BF01200129076
:104690001282120012921284120000011650FF0AB8
:0C46A00004E11294166A74EC22F012007F
:10BF0000E844F926000C160C2B0C3F0C520C640C68
:10BF1000760C860C960CA50CB30CC10CCF0CDC0C6B
:06BF2000E80CF40C000C1B
:00000001FF
